:020000040000FA
:0600000000008A017E2DC4
:08000800F0000308F1000A08F2
:10001000F2008A0183120313083081070B115C2060
:1000200019205C2072088A0071088300F00E700E9F
:10003000090087013F200310F70DF71E0800741C0C
:100040002D28203084001930F8008413000884170C
:100050008000840AF80B25287410A0308400013039
:10006000F700F90803193628F9030319F414FA0BF9
:1000700008006430FA00FB08031DFB0308004B2056
:100080004B204B204B204B20043085000030850056
:100090007708870008000530F800000DF600F60D1F
:1000A000F60D0030F60D0318023885000138850082
:1000B000F80B5128840A08000408F3067306F306B7
:1000C00084000800F5186B2875186E28751D080047
:1000D0007220800608007220800408007220FF3A17
:1000E000800508003F0884000310840D840D8407F8
:1000F000203084074008840700308A003E088207C9
:10010000103408340434023401341930C100203072
:1001100084008009840AC10B892808001F30A000D0
:10012000A100A200A300A400A500A600A700A800AB
:10013000A900AA00AB00AC00AD00AE00AF00B0005B
:10014000B100B200B300B400B500B600B700B8000B
:1001500008001F30F5188000751880017519800699
:1001600008006220BD20BD20BD20BD200800622007
:10017000C120C120C120C1200800840A840A840A49
:10018000840A840AF518800475198006751880059C
:100190000800C001BF01B120C00AB120C00AB120CF
:1001A000C00AB120C00AB1200800C0017220A920F5
:1001B000840AA920840AA920840AA920840AA920E3
:1001C0000800BF017220A92005308407A92005304E
:1001D0008407A92005308407A92005308407A920B9
:1001E00008003330C500450884000008840A840AEA
:1001F000840A840A840A8000C50345081F3A031D47
:10020000F328A001A101A201A301A4010800253047
:10021000C500450884000008840384038403840324
:1002200084038000C50A4508393A031D0929B40131
:10023000B501B601B701B80108003730C50045085F
:1002400084000008840A8000C50345081F3A031D86
:100250001F29A001A501AA01AF01B40108002130A6
:10026000C50045088400000884038000C50A4508CD
:10027000393A031D3129A401A901AE01B301B80126
:1002800008001930C500203084008012800C840AD8
:10029000C50B452908001930C50020308400031023
:1002A000800D840AC50B4F2908006220C703073060
:1002B000470503198329C71D61293E0A3E19030119
:1002C000BE00461C68290430BE08031D3E03BE0064
:1002D000471E6E293F0A3F190301BF00C71E75293B
:1002E0000430BF08031D3F03BF00471F7B29400A9E
:1002F00040190301C000C71F82290430C008031D34
:100300004003C000552908002008C2003408A0009E
:100310003808B4002408B8004208A4002108C2002C
:100320002F08A1003708AF002908B7004208A9002C
:100330002208C2002A08A2003608AA002E08B60029
:100340004208AE002308C2002508A3003508A50016
:100350003308B5004208B3002608C2003008A600E2
:100360003208B0002808B2004208A8002708C200DE
:100370002B08A7003108AB002D08B1004208AD00E2
:1003800008000A248A01C600C61B122A461B022A3C
:1003900001308A00CF30460703188A0A8200C1293B
:1003A000E42AE72A892AAB2AB12AAE2A232ABB2AC1
:1003B000BB2ABB2A6E2AC62AC62AC62AB42AB72A4C
:1003C000B92A882B8A2B102B0E2B122B142B162BB1
:1003D000182B3F2A442A4A2A502A542A582A5C2A8F
:1003E000A92A0A2B3D2ADB2BE22BE92BF02BF72B3A
:1003F000EA2AED2A622AA12BA32BAC2BFE2BB12BD0
:10040000BC2BC92B5E2302308A000A304607031832
:100410008A0A8200DC2AD42AE02AD82A7C2B7F2B65
:10042000F72AFB2A0A248A01C700461B662AC61A35
:10043000702A460C0F39031D1F2A4C23C129FF3E89
:10044000031D252A4C236220C129FF3E031D2A2AB1
:100450005521C129FF3E031D2F2AF5151A2BFF3EFA
:10046000031D342AF5111A2BFF3E0319FF2AFF3E04
:100470000319042BFF3E0319922A8421C129302439
:100480007220A9203724C1293024BF017220B12055
:100490003724C1293024C0017220B7203724C12954
:1004A0003024C9203724C1293024D5203724C1293C
:1004B0003024E1203724C1297220F41100050319EA
:1004C000F415C129F411051EF415C129C61A6823B3
:1004D00046081F39FD004708FC00C1297223C129C5
:1004E0005E234611460803197C2AFF3E03197F2A22
:1004F000FF3E0319832A112C47088000C1294708B1
:1005000012248000C129F41547080006031DF411C8
:10051000C129F41C892AF41074143D08F9007418D8
:100520008F2AC1296430FA004708FB00F411C7087C
:100530000319FB17FB080319C129051E972AC708D1
:100540000319FB17FB080319C129051A9F2AF41583
:10055000C1292B24C1290130F500C1290430F5003F
:10056000C1290230F500C12903018F20C1298E2045
:10057000C1298520C129460803393E3E8400043044
:100580008008031D00038000CF2AC12946080339D3
:100590003E3E8400800A0008053A03198001F415E4
:1005A0008008031DF411C1298003031DC129F02A0D
:1005B000800A031DC129F02AF415800BF411C1290A
:1005C000F415800FF411C129F41DC129F02AF41D7E
:1005D000F02AC129741EC129F02A741EF02AC129EB
:1005E0000A248A018039031D0A248A01C1290008CE
:1005F000C700F5151A2B0008C700F5111A2B643037
:10060000FA004708FB00C1296430FA0047081224A9
:10061000FB07C129FB08031DC129F02A1D21C1299F
:100620002F21C129F120C1290721C1294B21C1292D
:100630004121C1293024FF01203047023F39FE000B
:100640000310FE0DFE0DFE070318FF0A3E30FE07E5
:100650000318FF0A0430FF070530C7000430F519FE
:10066000BF00F51DC001722048238A01F5188004DF
:1006700075198006FF3A75188005FE0A0319FF0AEE
:10068000F519BF03F51DC00AC70B332B3724C12949
:100690007F088A007E0882004708BF000739C00033
:1006A000BF0CBF0C3F0C0739BF004708BE00460C0B
:1006B000BE0DBE0D3E0D0739BE00080046080739C5
:1006C000393E8400C60CC60C460C0739C60008002B
:1006D000430884007C088000840A7D088000040AA6
:1006E000C3000800430384000008FD0084030008E1
:1006F000FC000408C300080000088C23C12904087A
:10070000C7009823C5004708840045088000C12918
:10071000CD23C129D423C129C5004408840045083C
:100720008000C40A4408EB3AC9300319C400080029
:100730004408C93AEA30031D4403C4008400000899
:1007400008009823C1299823CE009823CF004E0893
:100750008C234F088C23C12998238C2345088C2394
:10076000C1299823CE009823CF004E088C234F0830
:100770008C234E088C23C1299823CE009823CF00C8
:100780009823D0004F088C234E088C2350088C23CC
:10079000C129982306248C23C1293E088C233F08B5
:1007A0008C2340088C2308009823C0009823BF00A6
:1007B0009823BE0008009823CD0098234D060624F8
:1007C0008C23C1299823CD0098234D0703248C2323
:1007D000C1299823CD0098234D0203248C23C129DD
:1007E0009823CD0098234D0506248C23C1299823F6
:1007F000CD0098234D0406248C23C1299823FF3A69
:1008000006248C23C129741203187416F4110319D9
:10081000F41508007D088A007C08FC0A0319FD0A0B
:100820008200112CCA000310C80CC90C031C1B2C1D
:10083000A130C806C9064808490703192B24CB0173
:10084000CC01CC17CA0C0318CB07CB0CCC0C031C67
:10085000222C4B080800010803192B2CC9000800A2
:100860003E08CE003F08CF004008D00008004E08E8
:10087000BE004F08BF005008C0000800003400341C
:1008800000340034003404340434043400340434B8
:100890000A340A340034003400340A341F340A3471
:1008A0001F340A340F3414340E3405341E34193412
:1008B0001A3404340B341334083414340D34123421
:1008C0000D340C340C340434083400340234043451
:1008D0000434043402340834043404340434083452
:1008E00015340E341F340E341534043404341F34DC
:1008F0000434043400340C340C340434083400342C
:1009000000341F34003400340034003400340C341C
:100910000C34013402340434083410340E341334EB
:10092000153419340E3404340C34043404340E34C5
:100930001E340134063408341F341E3401340E349E
:1009400001341E3406340A341F34023402341F3496
:1009500010341E3401341E34063408341E3411346D
:100960000E341F3402340434083408340E34113485
:100970000E3411340E340E3411340F3402340C346E
:100980000C340C3400340C340C340C3400340C347F
:100990000434083402340434083404340234003497
:1009A0001F3400341F340034083404340234043457
:1009B00008340E3411340234043404340E34153443
:1009C000173410340E3404340A341F341134113403
:1009D0001E3409340E3409341E340F3410341034EC
:1009E00010340F341E340934093409341E341F34D2
:1009F00010341E3410341F341F3410341E3410349D
:100A000010340F341034133411340F3411341134C2
:100A10001F34113411340E340434043404340E34CD
:100A200001340134013411340E34133414341834C5
:100A30001434133410341034103410341F3411347F
:100A40001B34153411341134113419341534133462
:100A500011340E341134113411340E341E34113467
:100A60001E34103410340C341234163412340D3455
:100A70001E3411341E34143412340F3410340E3436
:100A800001341E341F340434043404340434113467
:100A90001134113411340E341134113411340A3438
:100AA00004341134113415341B34113411340A3424
:100AB00004340A34113411340A3404340434043450
:100AC0001F340234043408341F340734043404342B
:100AD00004340734103408340434023401341C3430
:100AE0000434043404341C3404340A34113400341F
:100AF000003400340034003400341F346400073004
:100B0000990083160313910170308F000330810028
:100B1000D8308500103095008312031320308400F4
:100B20008417800184138001840A841F902D83160A
:100B30000313E030870083120313A030F300013069
:100B4000F700F4140530FD00B130FC00C930C400DA
:100B5000B930C3000130BD0008308100A0308B00E7
:100B6000C12921342B340134E6342134A43409342E
:100B7000A8343F345034E534BF34C534B63440343F
:100B80000234C634613440340234C634E434403470
:100B90000234C7341B3440340234C7348034403408
:100BA0000234C734AD3440340234C734E334403403
:100BB0000234C734F93440340234C834BE344034CB
:100BC0000234C934323440340234C93464344034D9
:100BD0000234C934AC3440340234C934D4344034DF
:100BE0000234CA34003440340234CA3483344034CA
:100BF0000234CA34B13440340234CA34B5344034D7
:100C00000234CA34B93440340234CB340F34403463
:100C10000234CB347C3440340234CB345D34403441
:100C20000234CB34C43440340234CC340B3440343A
:100C30000234CC345034C534BF342234C6341D346D
:100C40000B34A73404340534A0345034E634513422
:100C5000A0344934E6345134A0344334E6345134BA
:100C6000A0345034E6345134A0345234E634513494
:100C7000A0344F34E6345134A0344A34E63451348D
:100C8000A0344534E6345134A0344334E63451348E
:100C9000A0345434E6345134A0345334E63451345F
:100CA0000B34A43408340F34703403341434033454
:100CB00014340334143403341434A4342334033488
:100CC0000B34A43409348A3405348C3407340534A5
:100CD0000F348034003484341D348134043485343A
:100CE000153403340F348034403484341C3483345A
:100CF00021348034C43485341434823423340334AE
:100D00000F348034803484341B3481341934843477
:100D10005234803484348534133480341B34843426
:100D2000923403340F348034C03484341A34813420
:100D30001134843453348034443485341234803450
:100D400013348434933403340F34813400348434C2
:100D50005534803404348434953403340F3481346E
:100D60000134843454348234E4348034033484349D
:100D700094348234603403340F3481340234843444
:100D800053348034DC348534123480340234843477
:100D900093348034583484341A3403340F34813417
:100DA0000334843452348034D4348534133480345E
:100DB0000134843492348034503484341B3403340A
:100DC0002234C63468340B34A43401340F3405346F
:100DD000803400341E3403348A340A34A4340F348B
:100DE0000334AD340534AF340534A6340034A034B4
:100DF0000434A434053420340134C7340C34A6340C
:100E000004340434073409340534073403344834D3
:100E1000C7340134C7341734043407340D3405346F
:100E2000073403344834C7340C34C73417342234FD
:100E3000C634EE340B348A340A340F340334A1340C
:100E400000346134A4340334AD340534AE34053495
:100E5000AF340534A9340634683460346134243442
:100E60002C340234C73422346134B13400340234B7
:100E7000A5340034B13401340234A6340034B13422
:100E800002340234A7340034B13403340234A534BC
:100E90000434B13404340234A6340434B134053497
:100EA0000234A73404340534A0340534E734623402
:100EB0000434A0340534E734623403342234C734B4
:100EC00022340B3407340334B134003402340C348C
:100ED000B134013402340D34B134023402340E34EE
:100EE000B134033402340834B134043402340934E4
:100EF000B134053402340A344834C73462340B3414
:100F00000F3403340534A43423348234003483345E
:100F100000348334203483342434823424348234BF
:100F20000434833404348234203403348234493426
:100F300082344B348234593482345B348234C93441
:100F40008234CB348234D9348234DB340334823477
:100F5000923403340F34C6341D34A43432340F3485
:100F6000053482349234033482348A3482349A349D
:100F7000823452348234D234823491348234933481
:100F80000334803492341A341B341C348234513488
:100F90008234D334823453348234D1348234893429
:100FA00082348B3482344A348234CA348234993461
:100FB00082349B3482345A348234DA3403348A34AF
:100FC0000134C6341D34A43407348A340F34A634B3
:100FD00000340F3405341634E734F3340334223448
:100FE000C734EB340B34AD340534AF340534073437
:100FF0000B340F34A4340F340534803400341A34E5
:10100000803404341A3403341C34813400341C34E6
:101010000334A6340034A5340034A7340034073434
:10102000083407340A3407340C34073403340D34DD
:10103000B63400340134C8340B348034A2341E3446
:1010400004341A341C34033405341E340334173486
:101050000334173403341734033417340334163489
:101060000334163403340F348034103484340D3494
:10107000843445348534053484348534803459349B
:1010800084340B34843443348534033484348334DB
:1010900003348234A23403340F348234A23409344A
:1010A0001E34043482349A3403340D340F3405343E
:1010B0001E340334043482342034833420348334A3
:1010C000243482342434053482341834833418347C
:1010D00083341C3482341C3403340F348034A234FF
:1010E0001A341C3482346134823463348234E334FD
:1010F0008234E13482345834823419348234D8341E
:101100008334193483341B348234DC3482345C34C9
:1011100082341B34823410348334103483341434D6
:101120008234143403341734043482345A3482340D
:1011300099348234DA3482349B3482349A340534DC
:10114000823462348234A1348234E2348234A3346F
:101150008234A23403341734043482349A3405348C
:101160008234A2340334173403341734033417346D
:10117000033417340334173403340B340F34053479
:101180008234493482345134823489348234913403
:1011900082344A348234523482348A3482349234EF
:1011A0000334A4340B34A0341934A0340134A134F2
:1011B0000134A23401348A3405348C340A34AB341B
:1011C00005340234C834FC344B34C9340534AB34F0
:1011D00004340234C9340E344B34C9341734AB34BC
:1011E00003340234C93429344B34C9342034033431
:1011F0002234C834DF340B34B03400340234C83401
:10120000E73418344034C834E734B034033402349B
:10121000C834E73419345034C834E734B1340034B6
:101220000234C834EF3417344134C834EF34B134A5
:1012300003340234C834EF3416345134C834EF3434
:10124000B23400340234C834F73414344234C8346D
:10125000F734B23403340234C834F734153452341A
:10126000C834F7340F340534A4340C348A340A34C7
:101270008C3406341534803410341A3404348234F7
:1012800090340534033415348034003484341D34F0
:10129000043482349034053403341534803480347B
:1012A0001B340434823490340534033415348034D0
:1012B000203484342D34043482349034053403349F
:1012C0002234C9343A340B3405340F34A4340F3487
:1012D000813400341A3403341C340334803404342D
:1012E0001A3403341C3403348234083482340C340A
:1012F0008334083483340C3403348234103482341D
:101300001434833410348334143403348234183462
:1013100082341C348334183483341C3403348134D1
:1013200020341A3403341C340334803424341A3403
:1013300003341C34A43432340334A4340F341F3443
:1013400003341434033414340334143403341434A1
:10135000A434323403340B34A4340F3405340F3442
:101360008334243403340434103482340034E934B4
:10137000FC3482344934E934FC348234923403340A
:10138000103482340034E934FC3482344934E93492
:10139000FC340334103482340034E934FC34033434
:1013A0001034033405340B34A4340F3405340F34B3
:1013B0008234003403340434103483342434E93464
:1013C000FC348234DB34E934FC3482349234033428
:1013D000103483342434E934FC348234DB34E9348B
:1013E000FC340334103483342434E934FC340334BF
:1013F0001034033405340B341D341E341F340B34C5
:101400000F34A434093405348234943403348234E0
:101410009334823453348234D33482348B348234E0
:101420009B340334803492341A341B3482345A345B
:1014300082344A348234DA348234CA340334143481
:1014400082349434033414348234943403341434A2
:1014500082349434803400341F34043482340034B1
:10146000823420348334003483342034033405340C
:10147000143482349434803400341F3403340434FC
:1014800082349434823490340334823493348234FA
:101490009034823450348234D0348234883482346C
:1014A0009834033482349234803490341A341B34A8
:1014B00082345834823448348234D8348234C83444
:1014C000033405340F3482340034823420348334BE
:1014D0000034833420340334153403341534033496
:1014E00015340334153403340F3482344C348234CD
:1014F0005C348234CC348234DC3403340F348234B0
:10150000943403340B340F340534A4340E34803453
:101510000034E934FC3403340F3480344934E93482
:10152000FC3403340F3480349234E934FC34033413
:101530000F348034DB34E934FC3403340F34813429
:101540002434E934FC3403340B34A034053414342B
:10155000183417348334243403344834CA34A73459
:101560000B34EA34BD34CA34D034EA34BD34CA341E
:10157000FA34EA34BD34CA34E5340F340534AC34BB
:1015800008346434A4340834643425346C3480342E
:101590001034A03401348A3404348C3406340B34CF
:1015A0001C34033419346034663425346E34B63454
:1015B00004340234A034FF34B63400340234A0348E
:1015C00001342234CA34D0340B341B340334153480
:1015D0006034653425346D34B53404340234A034B9
:1015E000FF34B53400340234A03401342234CA3418
:1015F000E5340B341A34033415346034663425343E
:101600006E34B63404340234A034FF34B6340034BB
:101610000234A03401342234CA34FA340B34A434F2
:1016200007346434AC340A34643425346C341034F4
:101630000334043480342034EB344734EB344734FF
:10164000EB344734EB344734EB344734033403345E
:1016500080346134EB345234EB345234EB34523452
:10166000EB345234EB345234033403348234A23436
:10167000033482349A34033482349234033482340F
:101680008A34033482348234033403340B34843494
:101690000D3484344534853405348434853403343E
:1016A00009340B3484340B348434433485340334A8
:1016B00084348334033409340B34A4340A340F34AF
:1016C00003348A3403348C340434053483342434AE
:1016D000AB340334A4340A34EB348A34A4340534F0
:1016E0006434AC340C34643425346C34EB349734C7
:1016F0002234CB3476340B34A4341934103403340C
:10170000053483342434AB340434A4340A34EB3445
:1017100097340B34B334003402341F34B3340134FF
:1017200002341E34B334023402341D340B34EB342F
:10173000A834EB34A834EB34A834EB34A834EB34BD
:10174000B634EB34B634EB34B634EB34B6340B3455
:10175000B334003402341434B33401340234173453
:10176000B33402340234183403340B34B334003449
:1017700002341534B334013402341634B334023431
:101780000234193403340B34A03401346034A834E7
:1017900004346034253468340F340534A4340334FD
:1017A0006434AC340734643425346C34803400340D
:1017B0001A34EB34F7341534EC3401341534EB348B
:1017C000F7341534EC3401341534EB34F734143475
:1017D000EC3401341434EB34F7341434EC34013485
:1017E0001434EB34F7344834CB34DB340B34033467
:1017F00016340334163403341634033416340334E5
:101800000B340334173403341734033417340334DC
:10181000173403340B34A03403346034A834063452
:101820006034253468340F340534A434033464340C
:10183000AC340834643425346C348034003480345F
:1018400000341C34813400341C3403340F348034AD
:1018500048341C348034C8341C3403340F3480348E
:1018600090341C3403340F34803458341C348034A6
:10187000D8341C3403340F34803420341C34813485
:1018800020341C340334173403341734033417342E
:101890000334173403344834CC3426340B34213425
:1018A0000534A4340234A0340134A1340134A23408
:1018B0000134803492348A3405348C340A340F3441
:1018C00007340334EC3468342234CC345F340B34C2
:1018D0006034653425346D346134663425346E34B7
:1018E0006234673425346F34B53400340234EC3458
:1018F0009334B53404340234EC349734B6340034C1
:101900000234EC349B34B63404340234EC349F3467
:10191000B73400340234EC34A334B7340434023422
:10192000EC34A7340B34EC34AB3468340B34EC3483
:10193000B13468340B34EC34AB3469340B34EC34EC
:10194000B13469340B34EC34AB346A340B34EC34DA
:10195000B1346A340B34EC34BC34AB340234633409
:101960000B34EC34BC34AB340234B33401340234C1
:10197000A334FF3463340B34A43401346434AC3402
:0A1980000834643425346C340B3451
:02400E00E43399
:1042000020004C004500440020004300750062007F
:1042100065002000560031002E0030002E003200D4
:104220002000200061006E0069006D0061007400D4
:1042300069006F006E0073002000310033002D0014
:10424000300034002D0032003000300039002000F2
:104250002000700069006300700072006F006A0047
:1042600065006300740073002E006F007200670029
:104270002E0075006B00200020002800630029003C
:10428000200032003000300039002000500065006E
:104290007400650020004700720069006600660037
:0A42A000690074006800730020003C
:00000001FF
